:100000008316BF3087008601243098008130990024
:10001000831290309800FF3086003920003086002F
:100020008C1E102818191928981821281A088600DB
:1000300010281A08553086003920003086003920F3
:10004000192818121816AA308600392000308600A8
:1000500039202128A530A00000000000A00B2E2888
:1000600008006330A100000000002A20A10B352801
:1000700008006330A2006230A3000330A400000037
:100080003120A20B40282A20A30B4328A40B46288A
:02009000080066
:00000001FF
